 sw_emextG

 Timestamp is 540049ef (Fri Aug 29 17:37:51 2014)

 Preferred load address is 00100000

 Start         Length     Name                   Class
 0001:00000000 00011e48H .text                   CODE
 0001:00011e48 00000330H .text$yc                CODE
 0002:00000000 000057ecH .rdata                  DATA
 0002:000057ec 00000076H .rdata$debug            DATA
 0002:00005864 000000f8H .xdata                  DATA
 0002:0000595c 00000078H .idata$2                DATA
 0002:000059d4 00000014H .idata$3                DATA
 0002:000059e8 00000220H .idata$4                DATA
 0002:00005c08 00000372H .idata$6                DATA
 0002:00005f80 000000daH .edata                  DATA
 0003:00000000 00000220H .idata$5                DATA
 0003:00000220 00000004H .CRT$XCA                DATA
 0003:00000224 00000004H .CRT$XCAA               DATA
 0003:00000228 00000044H .CRT$XCU                DATA
 0003:0000026c 00000004H .CRT$XCZ                DATA
 0003:00000270 00000004H .CRT$XIA                DATA
 0003:00000274 00000004H .CRT$XIZ                DATA
 0003:00000278 00000004H .CRT$XPA                DATA
 0003:0000027c 00000004H .CRT$XPZ                DATA
 0003:00000280 00000004H .CRT$XTA                DATA
 0003:00000284 00000004H .CRT$XTZ                DATA
 0003:00000288 0000005cH .data                   DATA
 0003:000002e8 00001eb0H .bss                    DATA
 0004:00000000 00000630H .pdata                  DATA
 0005:00000000 000000a0H .rsrc$01                DATA
 0005:000000a0 000003d0H .rsrc$02                DATA

  Address         Publics by Value              Rva+Base       Lib:Object

 0000:00000000       ___safe_se_handler_count   00000000     <absolute>
 0000:00000000       ___safe_se_handler_table   00000000     <absolute>
 0001:00000000       ?SetDataTab@@YAXPAUHWND__@@@Z 00101000 f   data.obj
 0001:000001b4       ?InitializeData@@YAHPAUHWND__@@@Z 001011b4 f   data.obj
 0001:00000668       ?InitDataDlg@@YAHPAUHWND__@@@Z 00101668 f   data.obj
 0001:000006e8       ?OnMenuPopup@@YAHPAUHWND__@@I@Z 001016e8 f   data.obj
 0001:0000070c       ?RepairAndConfigureRegistry@@YAXXZ 0010170c f   data.obj
 0001:00000728       ?LaunchIOTA@@YAXXZ         00101728 f   data.obj
 0001:00000840       ?LaunchSWIOMADMClient@@YAXXZ 00101840 f   data.obj
 0001:0000091c       ?WndProcData@@YAHPAUHWND__@@IIJ@Z 0010191c f   data.obj
 0001:00000e54       ?CreateDataDlg@@YAHPAUHWND__@@@Z 00101e54 f   data.obj
 0001:0000110c       ?InitializeDatalist@@YAHPAUHWND__@@@Z 0010210c f   datalist.obj
 0001:00001398       ?InitDatalist@@YAHPAUHWND__@@@Z 00102398 f   datalist.obj
 0001:00001584       ?InitializeTabFromDatalistIndex@@YAHPAUHWND__@@K@Z 00102584 f   datalist.obj
 0001:00001778       ?OnDataListViewNotify@@YAJPAUHWND__@@J@Z 00102778 f   datalist.obj
 0001:00001afc       ?WndProcDatalist@@YAHPAUHWND__@@IIJ@Z 00102afc f   datalist.obj
 0001:00001cb0       ?CreateDatalistDlg@@YAHPAUHWND__@@@Z 00102cb0 f   datalist.obj
 0001:00001eac       ?SetStaticText@@YAXPAUHWND__@@@Z 00102eac f   location.obj
 0001:00001f80       ?SetLocationVal@@YAXPAUHWND__@@@Z 00102f80 f   location.obj
 0001:00002260       ?InitializeLocation@@YAHPAUHWND__@@@Z 00103260 f   location.obj
 0001:00002390       ?InitLocationDlg@@YAHPAUHWND__@@@Z 00103390 f   location.obj
 0001:00002418       ?WndProcLocation@@YAHPAUHWND__@@IIJ@Z 00103418 f   location.obj
 0001:0000286c       ?CreateLocatonDlg@@YAHPAUHWND__@@@Z 0010386c f   location.obj
 0001:00002b1c       IsDlgButtonChecked         00103b1c f i location.obj
 0001:00002b60       CheckDlgButton             00103b60 f i location.obj
 0001:00002bac       ?InitializePHSList@@YAHPAUHWND__@@@Z 00103bac f   phs_list.obj
 0001:00002e38       ?InitPhsList@@YAHPAUHWND__@@@Z 00103e38 f   phs_list.obj
 0001:00003024       ?InitializeTabFromPhsListIndex@@YAHPAUHWND__@@K@Z 00104024 f   phs_list.obj
 0001:00003374       ?OnListViewNotify@@YAJPAUHWND__@@J@Z 00104374 f   phs_list.obj
 0001:00003810       ?WndProcPhsList@@YAHPAUHWND__@@IIJ@Z 00104810 f   phs_list.obj
 0001:000039a4       ?CreatePHSListDlg@@YAHPAUHWND__@@@Z 001049a4 f   phs_list.obj
 0001:00003bac       ?ReadStrValue@@YAJPAUHKEY__@@PBG1QAGK@Z 00104bac f   ruim_call_ctrl.obj
 0001:00003cc8       ?WriteStrValue@@YAJPAUHKEY__@@PBG1QAGK@Z 00104cc8 f   ruim_call_ctrl.obj
 0001:00003e00       ?Init_RUIM_CALL_CTRL_Dlg@@YAHPAUHWND__@@@Z 00104e00 f   ruim_call_ctrl.obj
 0001:00003fe8       ?SendDialStr@@YAXPAG0@Z    00104fe8 f   ruim_call_ctrl.obj
 0001:0000415c       ?WndProc_RUIM_CALL_CTRL_Dlg@@YAHPAUHWND__@@IIJ@Z 0010515c f   ruim_call_ctrl.obj
 0001:000046f8       ?Create_RUIM_CALL_CTRL_Dlg@@YAHPAUHWND__@@@Z 001056f8 f   ruim_call_ctrl.obj
 0001:000049a8       ?Update_RUIM_CALL_CTRL_Dlg@@YAHPAUHWND__@@@Z 001059a8 f   ruim_call_ctrl.obj
 0001:00004e80       ??0ASCII@@QAA@PAG@Z        00105e80 f   ruim_pin.obj
 0001:00004f50       ??1ASCII@@QAA@XZ           00105f50 f   ruim_pin.obj
 0001:00004f7c       ??IASCII@@QAAPADXZ         00105f7c f   ruim_pin.obj
 0001:00004fa4       ??BASCII@@QAAPADXZ         00105fa4 f   ruim_pin.obj
 0001:00004fd4       ?HandlePIN1Action1@@YAHPAUHWND__@@@Z 00105fd4 f   ruim_pin.obj
 0001:00005924       ?HandlePIN1Action2@@YAHPAUHWND__@@@Z 00106924 f   ruim_pin.obj
 0001:00005c28       ?Update_RUIM_PIN_Dlg@@YAHPAUHWND__@@@Z 00106c28 f   ruim_pin.obj
 0001:00007060       ?Init_RUIM_PIN_Dlg@@YAHPAUHWND__@@@Z 00108060 f   ruim_pin.obj
 0001:000070f8       ?WndProc_RUIM_PIN_Dlg@@YAHPAUHWND__@@IIJ@Z 001080f8 f   ruim_pin.obj
 0001:0000738c       ?Create_RUIM_PIN_Dlg@@YAHPAUHWND__@@@Z 0010838c f   ruim_pin.obj
 0001:00007638       ?SetRoamingOption@@YAHPAK@Z 00108638 f   Sprint_roaming_option.obj
 0001:00007754       ?GetRoamingOption@@YAHPAK@Z 00108754 f   Sprint_roaming_option.obj
 0001:00007898       ?Init_SPRINT_ROAMING_OPTION_Dlg@@YAHPAUHWND__@@@Z 00108898 f   Sprint_roaming_option.obj
 0001:00007930       ?WndProc_SPRINT_ROAMING_OPTION_Dlg@@YAHPAUHWND__@@IIJ@Z 00108930 f   Sprint_roaming_option.obj
 0001:00007fa4       ?Create_SPRINT_ROAMING_OPTION_Dlg@@YAHPAUHWND__@@@Z 00108fa4 f   Sprint_roaming_option.obj
 0001:00008250       ?Update_SPRINT_ROAMING_OPTION_Dlg@@YAHPAUHWND__@@@Z 00109250 f   Sprint_roaming_option.obj
 0001:000084f8       ?GetInstanceHandle@@YAPAUHINSTANCE__@@XZ 001094f8 f   sw_emext.obj
 0001:00008518       ?GetResourceHandle@@YAPAUHINSTANCE__@@XZ 00109518 f   sw_emext.obj
 0001:00008538       ?GetCarrier@@YAKXZ         00109538 f   sw_emext.obj
 0001:00008558       ?InitializeGlobalVars@@YAXXZ 00109558 f   sw_emext.obj
 0001:00008620       ?InitializeRilValues@@YAXXZ 00109620 f   sw_emext.obj
 0001:0000865c       ?SetWindowTopMost@@YAJPAUHWND__@@@Z 0010965c f   sw_emext.obj
 0001:00008708       ?DebugOut@@YAXPBGZZ        00109708 f   sw_emext.obj
 0001:00008750       ??0PluginFactory@@QAA@XZ   00109750 f   sw_emext.obj
 0001:0000879c       ??1PluginFactory@@UAA@XZ   0010979c f   sw_emext.obj
 0001:000087bc       ?QueryInterface@PluginFactory@@UAAJABU_GUID@@PAPAX@Z 001097bc f   sw_emext.obj
 0001:00008870       ?CreateInstance@PluginFactory@@UAAJPAUIUnknown@@ABU_GUID@@PAPAX@Z 00109870 f   sw_emext.obj
 0001:000089b8       ?LockServer@PluginFactory@@UAAJH@Z 001099b8 f   sw_emext.obj
 0001:00008a18       DllGetClassObject          00109a18 f   sw_emext.obj
 0001:00008b50       DllCanUnloadNow            00109b50 f   sw_emext.obj
 0001:00008b94       DllRegisterServer          00109b94 f   sw_emext.obj
 0001:00008dfc       DllUnregisterServer        00109dfc f   sw_emext.obj
 0001:00008e80       ??0CSW_SysSettings@@QAA@XZ 00109e80 f   sw_emext.obj
 0001:00008f6c       ??1CSW_SysSettings@@QAA@XZ 00109f6c f   sw_emext.obj
 0001:00008fe8       ?QueryInterface@CSW_SysSettings@@UAAJABU_GUID@@PAPAX@Z 00109fe8 f   sw_emext.obj
 0001:000092bc       ?PropPageProc@@YAHPAUHWND__@@IIJ@Z 0010a2bc f   sw_emext.obj
 0001:00009e14       ?PropSheetCallback@@YAIPAUHWND__@@IPAU_PROPSHEETPAGEW@@@Z 0010ae14 f   sw_emext.obj
 0001:00009e7c       ?AddPages@CSW_SysSettings@@UAAJP6AHPAU_PSP@@J@ZJ@Z 0010ae7c f   sw_emext.obj
 0001:0000a6e8       ?ReplacePage@CSW_SysSettings@@UAAJIP6AHPAU_PSP@@J@ZJ@Z 0010b6e8 f   sw_emext.obj
 0001:0000a75c       ?SWDialExtERIWndProc@@YAJPAUHWND__@@IIJ@Z 0010b75c f   sw_emext.obj
 0001:0000a920       ?CreateERIWindow@@YAJPAUHWND__@@PAPAU1@@Z 0010b920 f   sw_emext.obj
 0001:0000aaf0       ?ResetPowerState@@YAHXZ    0010baf0 f   sw_emext.obj
 0001:0000ab38       ?CheckPowerstate@@YAHXZ    0010bb38 f   sw_emext.obj
 0001:0000ac18       ?IsUserInActivecall@@YAHXZ 0010bc18 f   sw_emext.obj
 0001:0000ac88       ?GetStatus@@YAXXZ          0010bc88 f   sw_emext.obj
 0001:0000acb4       ?SetLocationMode@@YAHK@Z   0010bcb4 f   sw_emext.obj
 0001:0000ad04       ?SetPreferredPrivacyMode@@YAHK@Z 0010bd04 f   sw_emext.obj
 0001:0000ad54       ?SetRoamingMode@@YAHK@Z    0010bd54 f   sw_emext.obj
 0001:0000ada4       ?GetRoamingMode@@YAHXZ     0010bda4 f   sw_emext.obj
 0001:0000ae00       ?GetLocationStatus@@YAHXZ  0010be00 f   sw_emext.obj
 0001:0000ae5c       ?GetRoamStatus@@YAHXZ      0010be5c f   sw_emext.obj
 0001:0000aeb8       ?GetPreferredPrivacyMode@@YAHXZ 0010beb8 f   sw_emext.obj
 0001:0000af14       ?LaunchAAM@@YAKPAX@Z       0010bf14 f   sw_emext.obj
 0001:0000afdc       DllMain                    0010bfdc f   sw_emext.obj
 0001:0000b0d4       ?Initialize@CSW_SysSettings@@UAAJPFBU_ITEMIDLIST@@PAUIDataObject@@PAUHKEY__@@@Z 0010c0d4 f   sw_emext.obj
 0001:0000b1c4       ?SetSite@CSW_SysSettings@@UAAJPAUIUnknown@@@Z 0010c1c4 f   sw_emext.obj
 0001:0000b2b8       ?GetSite@CSW_SysSettings@@UAAJABU_GUID@@PAPAX@Z 0010c2b8 f   sw_emext.obj
 0001:0000b38c       ?GetTypeInfoCount@CSW_SysSettings@@UAAJPAI@Z 0010c38c f   sw_emext.obj
 0001:0000b3bc       ?GetTypeInfo@CSW_SysSettings@@UAAJIKPAPAUITypeInfo@@@Z 0010c3bc f   sw_emext.obj
 0001:0000b3e4       ?GetIDsOfNames@CSW_SysSettings@@UAAJABU_GUID@@PAPAGIKPAJ@Z 0010c3e4 f   sw_emext.obj
 0001:0000b414       ?Invoke@CSW_SysSettings@@UAAJJABU_GUID@@KGPAUtagDISPPARAMS@@PAUtagVARIANT@@PAUtagEXCEPINFO@@PAI@Z 0010c414 f   sw_emext.obj
 0001:0000b7b0       LoadOemDataIcon            0010c7b0 f   sw_emext.obj
 0001:0000ba40       FreeOemDataIcon            0010ca40 f   sw_emext.obj
 0001:0000bb98       ?AddRef@PluginFactory@@UAAKXZ 0010cb98 f i sw_emext.obj
 0001:0000bbe0       ?Release@PluginFactory@@UAAKXZ 0010cbe0 f i sw_emext.obj
 0001:0000bc9c       ??_GPluginFactory@@UAAPAXI@Z 0010cc9c f i sw_emext.obj
 0001:0000bc9c       ??_EPluginFactory@@UAAPAXI@Z 0010cc9c f i sw_emext.obj
 0001:0000bcdc       ??0IClassFactory@@QAA@XZ   0010ccdc f i sw_emext.obj
 0001:0000bd08       ??0IUnknown@@QAA@XZ        0010cd08 f i sw_emext.obj
 0001:0000bd2c       ??8@YAHABU_GUID@@0@Z       0010cd2c f i sw_emext.obj
 0001:0000bd84       ?Reset@CSW_SysSettings@@QAAXXZ 0010cd84 f i sw_emext.obj
 0001:0000bde4       ?AddRef@CSW_SysSettings@@UAAKXZ 0010cde4 f i sw_emext.obj
 0001:0000be2c       ?Release@CSW_SysSettings@@UAAKXZ 0010ce2c f i sw_emext.obj
 0001:0000bed4       ??_GCSW_SysSettings@@QAAPAXI@Z 0010ced4 f i sw_emext.obj
 0001:0000bf14       ??0IObjectWithSite@@QAA@XZ 0010cf14 f i sw_emext.obj
 0001:0000bf50       ??0IShellExtInit@@QAA@XZ   0010cf50 f i sw_emext.obj
 0001:0000bf8c       ??0IDispatch@@QAA@XZ       0010cf8c f i sw_emext.obj
 0001:0000bfb8       ??0IShellPropSheetExt@@QAA@XZ 0010cfb8 f i sw_emext.obj
 0001:0000bff4       ?IsEqualGUID@@YAHABU_GUID@@0@Z 0010cff4 f i sw_emext.obj
 0001:0000c04c       ??9@YAHABU_GUID@@0@Z       0010d04c f i sw_emext.obj
 0001:0000c0a0       ?AddRef@CSW_SysSettings@@W7AAKXZ 0010d0a0 f i sw_emext.obj
 0001:0000c0a8       ?AddRef@CSW_SysSettings@@WM@AAKXZ 0010d0a8 f i sw_emext.obj
 0001:0000c0b0       ?QueryInterface@CSW_SysSettings@@W3AAJABU_GUID@@PAPAX@Z 0010d0b0 f i sw_emext.obj
 0001:0000c0b8       ?QueryInterface@CSW_SysSettings@@W7AAJABU_GUID@@PAPAX@Z 0010d0b8 f i sw_emext.obj
 0001:0000c0c0       ?Release@CSW_SysSettings@@W3AAKXZ 0010d0c0 f i sw_emext.obj
 0001:0000c0c8       ?QueryInterface@CSW_SysSettings@@WM@AAJABU_GUID@@PAPAX@Z 0010d0c8 f i sw_emext.obj
 0001:0000c0d0       ?Release@CSW_SysSettings@@W7AAKXZ 0010d0d0 f i sw_emext.obj
 0001:0000c0d8       ?Release@CSW_SysSettings@@WM@AAKXZ 0010d0d8 f i sw_emext.obj
 0001:0000c0e0       ?AddRef@CSW_SysSettings@@W3AAKXZ 0010d0e0 f i sw_emext.obj
 0001:0000c0f0       ?PopulateVZWSysTab@@YAXPAUHWND__@@@Z 0010d0f0 f   syssettings.obj
 0001:0000c63c       ?PopulatePCSSysTab@@YAXPAUHWND__@@@Z 0010d63c f   syssettings.obj
 0001:0000ca34       ?PopulateGenSysTab@@YAXPAUHWND__@@@Z 0010da34 f   syssettings.obj
 0001:0000cf8c       ?SetPreferredPrivacyMode@@YAXPAUHWND__@@@Z 0010df8c f   syssettings.obj
 0001:0000d038       ?SetRoamingVal@@YAXPAUHWND__@@@Z 0010e038 f   syssettings.obj
 0001:0000d39c       ?InitializeSysSettings@@YAHPAUHWND__@@@Z 0010e39c f   syssettings.obj
 0001:0000d59c       ?InitSysSettingsDlg@@YAHPAUHWND__@@@Z 0010e59c f   syssettings.obj
 0001:0000d61c       ?WndProcSysSettings@@YAHPAUHWND__@@IIJ@Z 0010e61c f   syssettings.obj
 0001:0000dad8       ?CreateSysSettingDlg@@YAHPAUHWND__@@@Z 0010ead8 f   syssettings.obj
 0001:0000dd8c       ?InitializeVersionInfoDlg@@YAHPAUHWND__@@AAUtagRILVERNOINFO@@@Z 0010ed8c f   versioninfo.obj
 0001:0000ec90       ?InitVersionInfoDlg@@YAHPAUHWND__@@@Z 0010fc90 f   versioninfo.obj
 0001:0000ed40       ?WndProcVersionInfoDlg@@YAHPAUHWND__@@IIJ@Z 0010fd40 f   versioninfo.obj
 0001:0000ef28       ?CreateVersionInfoDlg@@YAHPAUHWND__@@@Z 0010ff28 f   versioninfo.obj
 0001:0000f1d4       DestroyPropertySheetPage   001101d4 f   commctrl:commctrl.dll
 0001:0000f1e4       CreatePropertySheetPageW   001101e4 f   commctrl:commctrl.dll
 0001:0000f1f4       UpdateWindow               001101f4 f   coredll:COREDLL.dll
 0001:0000f204       EnableWindow               00110204 f   coredll:COREDLL.dll
 0001:0000f214       GetDlgItem                 00110214 f   coredll:COREDLL.dll
 0001:0000f224       ShowWindow                 00110224 f   coredll:COREDLL.dll
 0001:0000f234       SetWindowTextW             00110234 f   coredll:COREDLL.dll
 0001:0000f244       wcscat                     00110244 f   coredll:COREDLL.dll
 0001:0000f254       LoadStringW                00110254 f   coredll:COREDLL.dll
 0001:0000f264       MessageBoxW                00110264 f   coredll:COREDLL.dll
 0001:0000f274       GetLastError               00110274 f   coredll:COREDLL.dll
 0001:0000f284       CreateProcessW             00110284 f   coredll:COREDLL.dll
 0001:0000f294       SetFocus                   00110294 f   coredll:COREDLL.dll
 0001:0000f2a4       EndDialog                  001102a4 f   coredll:COREDLL.dll
 0001:0000f2b4       DialogBoxIndirectParamW    001102b4 f   coredll:COREDLL.dll
 0001:0000f2c4       LoadResource               001102c4 f   coredll:COREDLL.dll
 0001:0000f2d4       FindResourceW              001102d4 f   coredll:COREDLL.dll
 0001:0000f2e4       swprintf                   001102e4 f   coredll:COREDLL.dll
 0001:0000f2f4       RegisterClassW             001102f4 f   coredll:COREDLL.dll
 0001:0000f304       GetStockObject             00110304 f   coredll:COREDLL.dll
 0001:0000f314       memset                     00110314 f   coredll:COREDLL.dll
 0001:0000f324       RegisterWindowMessageW     00110324 f   coredll:COREDLL.dll
 0001:0000f334       SetWindowPos               00110334 f   coredll:COREDLL.dll
 0001:0000f344       GetClientRect              00110344 f   coredll:COREDLL.dll
 0001:0000f354       SendMessageW               00110354 f   coredll:COREDLL.dll
 0001:0000f364       SendDlgItemMessageW        00110364 f   coredll:COREDLL.dll
 0001:0000f374       RegCloseKey                00110374 f   coredll:COREDLL.dll
 0001:0000f384       NKDbgPrintfW               00110384 f   coredll:COREDLL.dll
 0001:0000f394       RegQueryValueExW           00110394 f   coredll:COREDLL.dll
 0001:0000f3a4       RegOpenKeyExW              001103a4 f   coredll:COREDLL.dll
 0001:0000f3b4       RegSetValueExW             001103b4 f   coredll:COREDLL.dll
 0001:0000f3c4       RegCreateKeyExW            001103c4 f   coredll:COREDLL.dll
 0001:0000f3d4       wsprintfW                  001103d4 f   coredll:COREDLL.dll
 0001:0000f3e4       _isctype                   001103e4 f   coredll:COREDLL.dll
 0001:0000f3f4       wcslen                     001103f4 f   coredll:COREDLL.dll
 0001:0000f404       GetWindowTextW             00110404 f   coredll:COREDLL.dll
 0001:0000f414       KillTimer                  00110414 f   coredll:COREDLL.dll
 0001:0000f424       SetTimer                   00110424 f   coredll:COREDLL.dll
 0001:0000f434       malloc                     00110434 f   coredll:COREDLL.dll
 0001:0000f444       WideCharToMultiByte        00110444 f   coredll:COREDLL.dll
 0001:0000f454       free                       00110454 f   coredll:COREDLL.dll
 0001:0000f464       strcpy                     00110464 f   coredll:COREDLL.dll
 0001:0000f474       memcpy                     00110474 f   coredll:COREDLL.dll
 0001:0000f484       LoadLibraryW               00110484 f   coredll:COREDLL.dll
 0001:0000f494       GetWindowRect              00110494 f   coredll:COREDLL.dll
 0001:0000f4a4       SetWindowLongW             001104a4 f   coredll:COREDLL.dll
 0001:0000f4b4       GetWindowLongW             001104b4 f   coredll:COREDLL.dll
 0001:0000f4c4       OutputDebugStringW         001104c4 f   coredll:COREDLL.dll
 0001:0000f4d4       wvsprintfW                 001104d4 f   coredll:COREDLL.dll
 0001:0000f4e4       ??3@YAXPAX@Z               001104e4 f   coredll:COREDLL.dll
 0001:0000f4f4       ??2@YAPAXI@Z               001104f4 f   coredll:COREDLL.dll
 0001:0000f504       memcmp                     00110504 f   coredll:COREDLL.dll
 0001:0000f514       GetModuleFileNameW         00110514 f   coredll:COREDLL.dll
 0001:0000f524       GetModuleHandleW           00110524 f   coredll:COREDLL.dll
 0001:0000f534       RegDeleteKeyW              00110534 f   coredll:COREDLL.dll
 0001:0000f544       _purecall                  00110544 f   coredll:COREDLL.dll
 0001:0000f554       PostMessageW               00110554 f   coredll:COREDLL.dll
 0001:0000f564       RemoveProp                 00110564 f   coredll:COREDLL.dll
 0001:0000f574       GetActiveWindow            00110574 f   coredll:COREDLL.dll
 0001:0000f584       wcscpy                     00110584 f   coredll:COREDLL.dll
 0001:0000f594       DefWindowProcW             00110594 f   coredll:COREDLL.dll
 0001:0000f5a4       EndPaint                   001105a4 f   coredll:COREDLL.dll
 0001:0000f5b4       DrawTextW                  001105b4 f   coredll:COREDLL.dll
 0001:0000f5c4       ExtTextOutW                001105c4 f   coredll:COREDLL.dll
 0001:0000f5d4       BeginPaint                 001105d4 f   coredll:COREDLL.dll
 0001:0000f5e4       InvalidateRect             001105e4 f   coredll:COREDLL.dll
 0001:0000f5f4       CreateWindowExW            001105f4 f   coredll:COREDLL.dll
 0001:0000f604       Sleep                      00110604 f   coredll:COREDLL.dll
 0001:0000f614       CreateThread               00110614 f   coredll:COREDLL.dll
 0001:0000f624       LoadIconW                  00110624 f   coredll:COREDLL.dll
 0001:0000f634       DestroyIcon                00110634 f   coredll:COREDLL.dll
 0001:0000f644       wcsncpy                    00110644 f   coredll:COREDLL.dll
 0001:0000f654       __rt_sdiv                  00110654 f   coredll:COREDLL.dll
 0001:0000f664       SHInitDialog               00110664 f   aygshell:AYGSHELL.dll
 0001:0000f674       SHCreateMenuBar            00110674 f   aygshell:AYGSHELL.dll
 0001:0000f684       GetLogoTestReg             00110684 f   sw_utilityG:sw_utilityG.dll
 0001:0000f694       ?SetConnectionProfile@@YAJXZ 00110694 f   sw_utilityG:sw_utilityG.dll
 0001:0000f6a4       ?LogC@@YAXPBGZZ            001106a4 f   sw_utilityG:sw_utilityG.dll
 0001:0000f6b4       ?WriteLog@@YAXKPBGZZ       001106b4 f   sw_utilityG:sw_utilityG.dll
 0001:0000f6c4       ?LogStoreFileLine@@YAXPAGH@Z 001106c4 f   sw_utilityG:sw_utilityG.dll
 0001:0000f6d4       GetOMADMConfig             001106d4 f   sw_utilityG:sw_utilityG.dll
 0001:0000f6e4       ?RelayoutDialog@@YAHPAUHINSTANCE__@@PAUHWND__@@PBG@Z 001106e4 f   sw_utilityG:sw_utilityG.dll
 0001:0000f6f4       ?InWideMode@@YAHXZ         001106f4 f   sw_utilityG:sw_utilityG.dll
 0001:0000f704       SetEquipmentState          00110704 f   sw_utilityG:sw_utilityG.dll
 0001:0000f714       ?SetWaitCursor@@YAXXZ      00110714 f   sw_utilityG:sw_utilityG.dll
 0001:0000f724       ?SetNormalCursor@@YAXXZ    00110724 f   sw_utilityG:sw_utilityG.dll
 0001:0000f734       ?GetCarrierIndex@@YAKXZ    00110734 f   sw_utilityG:sw_utilityG.dll
 0001:0000f744       ?GetProductFeatures@@YAHAAK@Z 00110744 f   sw_utilityG:sw_utilityG.dll
 0001:0000f754       ?LogW@@YAXPBGZZ            00110754 f   sw_utilityG:sw_utilityG.dll
 0001:0000f764       GetRilStatus               00110764 f   sw_utilityG:sw_utilityG.dll
 0001:0000f774       ModSetLocationMode         00110774 f   sw_utilityG:sw_utilityG.dll
 0001:0000f784       ModSetPreferredPrivacyMode 00110784 f   sw_utilityG:sw_utilityG.dll
 0001:0000f794       ModSetRoamingMode          00110794 f   sw_utilityG:sw_utilityG.dll
 0001:0000f7a4       ModGetRoamingMode          001107a4 f   sw_utilityG:sw_utilityG.dll
 0001:0000f7b4       ModGetLocationStatus       001107b4 f   sw_utilityG:sw_utilityG.dll
 0001:0000f7c4       ModGetRoamStatus           001107c4 f   sw_utilityG:sw_utilityG.dll
 0001:0000f7d4       ModGetPreferredPrivacyMode 001107d4 f   sw_utilityG:sw_utilityG.dll
 0001:0000f7e4       ?LogV@@YAXPBGZZ            001107e4 f   sw_utilityG:sw_utilityG.dll
 0001:0000f7f4       ?GetVerInfo@@YAPAGPAUHINSTANCE__@@@Z 001107f4 f   sw_utilityG:sw_utilityG.dll
 0001:0000f804       ?InitLog@@YAXPAUHINSTANCE__@@@Z 00110804 f   sw_utilityG:sw_utilityG.dll
 0001:0000f814       ?GetCallGuardReg@@YAKXZ    00110814 f   sw_utilityG:sw_utilityG.dll
 0001:0000f824       ?SetAutoUpdateTime@@YAXH@Z 00110824 f   sw_utilityG:sw_utilityG.dll
 0001:0000f834       ?GetAutoUpdateTimeUI@@YAKXZ 00110834 f   sw_utilityG:sw_utilityG.dll
 0001:0000f844       ?GetAutoUpdateTime@@YAKXZ  00110844 f   sw_utilityG:sw_utilityG.dll
 0001:0000f854       ?SetCallGuardReg@@YAXK@Z   00110854 f   sw_utilityG:sw_utilityG.dll
 0001:0000f864       GetVersionInfo             00110864 f   sw_utilityG:sw_utilityG.dll
 0001:0000f874       GetRTREConfig              00110874 f   gobiapi:GobiApi.dll
 0001:0000f884       UIMUnblockPIN              00110884 f   gobiapi:GobiApi.dll
 0001:0000f894       UIMSetPINProtection        00110894 f   gobiapi:GobiApi.dll
 0001:0000f8a4       UIMVerifyPIN               001108a4 f   gobiapi:GobiApi.dll
 0001:0000f8b4       UIMChangePIN               001108b4 f   gobiapi:GobiApi.dll
 0001:0000f8c4       UIMGetCardStatus           001108c4 f   gobiapi:GobiApi.dll
 0001:0000f8d4       SetCDMANetworkParameters   001108d4 f   gobiapi:GobiApi.dll
 0001:0000f8e4       GetCDMANetworkParameters   001108e4 f   gobiapi:GobiApi.dll
 0001:0000f8f4       SwiSetDeviceRemovalCallback 001108f4 f   gobiapi:GobiApi.dll
 0001:0000f904       QCWWANConnect              00110904 f   gobiapi:GobiApi.dll
 0001:0000f914       QCWWANDisconnect           00110914 f   gobiapi:GobiApi.dll
 0001:0000f924       tapiRequestMakeCallW       00110924 f   cellcore:cellcore.dll
 0001:0000f934       _DllMainCRTStartup         00110934 f   corelibc:pegdmain.obj
 0001:0000f9cc       __security_check_cookie    001109cc     corelibc:armsecgs.obj
 0001:0000f9e0       __gsfailure                001109e0     corelibc:armsecgs.obj
 0001:0000fa24       GetCurrentProcess          00110a24 f i corelibc:crt0dat.obj
 0001:0000fa60       _cinit                     00110a60 f   corelibc:crt0dat.obj
 0001:0000fbd0       exit                       00110bd0 f   corelibc:crt0dat.obj
 0001:0000fbe8       _exit                      00110be8 f   corelibc:crt0dat.obj
 0001:0000fc00       _cexit                     00110c00 f   corelibc:crt0dat.obj
 0001:0000fc1c       _c_exit                    00110c1c f   corelibc:crt0dat.obj
 0001:0000fc68       __security_init_cookie     00110c68 f   corelibc:seccinit.obj
 0001:0000fcb8       __GSHandlerCheckCommon     00110cb8 f   LIBCMTD:gshandler.obj
 0001:0000fd00       __GSHandlerCheck           00110d00 f   LIBCMTD:gshandler.obj
 0001:0000fd30       __InternalCxxFrameHandler  00110d30 f   LIBCMTD:frame_ce.obj
 0001:0000ff0c       __CxxFrameHandler3         00110f0c f   LIBCMTD:frame_ce.obj
 0001:000106e8       __FrameUnwindToState       001116e8 f   LIBCMTD:frame_ce.obj
 0001:00011494       ?_DestructExceptionObject@@YAXPAUEHExceptionRecord@@E@Z 00112494 f   LIBCMTD:frame_ce.obj
 0001:000115e4       ?_OffsetToAddress@@YAPAXHPAKK@Z 001125e4 f   LIBCMTD:frame_ce.obj
 0001:00011670       ?FindFrameInfo@@YAPAU_FrameInfo@@PAK@Z 00112670 f   LIBCMTD:frame_ce.obj
 0001:000116f8       ?FindCatchFrameInfo@@YAPAU_FrameInfo@@PAK@Z 001126f8 f   LIBCMTD:frame_ce.obj
 0001:0001177c       ?_GetRangeOfTrysToCheck@@YAPBU_s_TryBlockMapEntry@@PBU_s_FuncInfo@@HHPAI1@Z 0011277c f   LIBCMTD:frame_ce.obj
 0001:00011874       __GSHandlerCheck_EH        00112874 f   LIBCMTD:gshandlereh.obj
 0001:00011908       GetCRTStorage              00112908 f   LIBCMTD:corecrt.obj
 0001:00011a18       TlsAlloc                   00112a18 f i LIBCMTD:corecrt.obj
 0001:00011a54       TlsFree                    00112a54 f i LIBCMTD:corecrt.obj
 0001:00011a98       ?FindFrameForUnwind@@YAPAKPAKPBU_s_FuncInfo@@@Z 00112a98 f   LIBCMTD:mdframe_arm.obj
 0001:00011b30       ?FindCatchFrame@@YAPAKPAKK@Z 00112b30 f   LIBCMTD:mdframe_arm.obj
 0001:00011bc8       ?AdjustFrameForCatch@@YAPAKPAKPBU_s_FuncInfo@@@Z 00112bc8 f   LIBCMTD:mdframe_arm.obj
 0001:00011c68       ?GetCurrentState@@YAHPAKPAU_DISPATCHER_CONTEXT@@PBU_s_FuncInfo@@@Z 00112c68 f   LIBCMTD:ehstate_arm_mips.obj
 0001:00011d44       _CallSettingFrame          00112d44     LIBCMTD:handlers_arm.obj
 0001:00011d88       __report_gsfailure         00112d88 f   coredll:COREDLL.dll
 0001:00011d98       LocalFree                  00112d98 f   coredll:COREDLL.dll
 0001:00011da8       __security_gen_cookie      00112da8 f   coredll:COREDLL.dll
 0001:00011db8       strcmp                     00112db8 f   coredll:COREDLL.dll
 0001:00011dc8       __C_specific_handler       00112dc8 f   coredll:COREDLL.dll
 0001:00011dd8       ?terminate@std@@YAXXZ      00112dd8 f   coredll:COREDLL.dll
 0001:00011de8       memmove                    00112de8 f   coredll:COREDLL.dll
 0001:00011df8       TlsSetValue                00112df8 f   coredll:COREDLL.dll
 0001:00011e08       LocalAlloc                 00112e08 f   coredll:COREDLL.dll
 0001:00011e18       TlsGetValue                00112e18 f   coredll:COREDLL.dll
 0001:00011e28       InterlockedCompareExchange 00112e28 f   coredll:COREDLL.dll
 0001:00011e38       TlsCall                    00112e38 f   coredll:COREDLL.dll
 0002:00003a60       CLSID_SWEMEXTCPL           00117a60     sw_emext.obj
 0002:00003a70       IID_ITPCSettingsFullCustomCPL 00117a70     sw_emext.obj
 0002:00003a80       IID_IObjectWithSite        00117a80     sw_emext.obj
 0002:00003a90       GUID_NULL                  00117a90     sw_emext.obj
 0002:00003aa0       IID_IUnknown               00117aa0     sw_emext.obj
 0002:00003ab0       IID_IClassFactory          00117ab0     sw_emext.obj
 0002:00003ac0       IID_IMalloc                00117ac0     sw_emext.obj
 0002:00003ad0       IID_IMarshal               00117ad0     sw_emext.obj
 0002:00003ae0       IID_IRpcChannel            00117ae0     sw_emext.obj
 0002:00003af0       IID_IRpcStub               00117af0     sw_emext.obj
 0002:00003b00       IID_IStubManager           00117b00     sw_emext.obj
 0002:00003b10       IID_IRpcProxy              00117b10     sw_emext.obj
 0002:00003b20       IID_IProxyManager          00117b20     sw_emext.obj
 0002:00003b30       IID_IPSFactory             00117b30     sw_emext.obj
 0002:00003b40       IID_ILockBytes             00117b40     sw_emext.obj
 0002:00003b50       IID_IStorage               00117b50     sw_emext.obj
 0002:00003b60       IID_IStream                00117b60     sw_emext.obj
 0002:00003b70       IID_IEnumSTATSTG           00117b70     sw_emext.obj
 0002:00003b80       IID_IBindCtx               00117b80     sw_emext.obj
 0002:00003b90       IID_IMoniker               00117b90     sw_emext.obj
 0002:00003ba0       IID_IRunningObjectTable    00117ba0     sw_emext.obj
 0002:00003bb0       IID_IInternalMoniker       00117bb0     sw_emext.obj
 0002:00003bc0       IID_IRootStorage           00117bc0     sw_emext.obj
 0002:00003bd0       IID_IDfReserved1           00117bd0     sw_emext.obj
 0002:00003be0       IID_IDfReserved2           00117be0     sw_emext.obj
 0002:00003bf0       IID_IDfReserved3           00117bf0     sw_emext.obj
 0002:00003c00       IID_IMessageFilter         00117c00     sw_emext.obj
 0002:00003c10       CLSID_StdMarshal           00117c10     sw_emext.obj
 0002:00003c20       IID_IStdMarshalInfo        00117c20     sw_emext.obj
 0002:00003c30       IID_IExternalConnection    00117c30     sw_emext.obj
 0002:00004eac       ??_7PluginFactory@@6B@     00118eac     sw_emext.obj
 0002:00004ec4       ??_7CSW_SysSettings@@6BIShellPropSheetExt@@@ 00118ec4     sw_emext.obj
 0002:00004ed8       ??_7CSW_SysSettings@@6BIDispatch@@@ 00118ed8     sw_emext.obj
 0002:00004ef4       ??_7CSW_SysSettings@@6BIShellExtInit@@@ 00118ef4     sw_emext.obj
 0002:00004f04       ??_7CSW_SysSettings@@6BIObjectWithSite@@@ 00118f04     sw_emext.obj
 0002:00004f18       ??_7IObjectWithSite@@6B@   00118f18     sw_emext.obj
 0002:00004f2c       ??_7IShellExtInit@@6B@     00118f2c     sw_emext.obj
 0002:00004f3c       ??_7IShellPropSheetExt@@6B@ 00118f3c     sw_emext.obj
 0002:000057bc       IID_IShellPropSheetExt     001197bc     uuid:shguids_guid29.obj
 0002:000057cc       IID_IDispatch              001197cc     uuid:oaidl_i_guid4.obj
 0002:000057dc       IID_IShellExtInit          001197dc     uuid:shguids_guid28.obj
 0002:0000595c       __IMPORT_DESCRIPTOR_commctrl 0011995c     commctrl:commctrl.dll
 0002:00005970       __IMPORT_DESCRIPTOR_COREDLL 00119970     coredll:COREDLL.dll
 0002:00005984       __IMPORT_DESCRIPTOR_AYGSHELL 00119984     aygshell:AYGSHELL.dll
 0002:00005998       __IMPORT_DESCRIPTOR_sw_utilityG 00119998     sw_utilityG:sw_utilityG.dll
 0002:000059ac       __IMPORT_DESCRIPTOR_GobiApi 001199ac     gobiapi:GobiApi.dll
 0002:000059c0       __IMPORT_DESCRIPTOR_cellcore 001199c0     cellcore:cellcore.dll
 0002:000059d4       __NULL_IMPORT_DESCRIPTOR   001199d4     commctrl:commctrl.dll
 0003:00000000       __imp_SHInitDialog         0011b000     aygshell:AYGSHELL.dll
 0003:00000004       __imp_SHCreateMenuBar      0011b004     aygshell:AYGSHELL.dll
 0003:00000008       \177AYGSHELL_NULL_THUNK_DATA 0011b008     aygshell:AYGSHELL.dll
 0003:0000000c       __imp_UpdateWindow         0011b00c     coredll:COREDLL.dll
 0003:00000010       __imp_EnableWindow         0011b010     coredll:COREDLL.dll
 0003:00000014       __imp_GetDlgItem           0011b014     coredll:COREDLL.dll
 0003:00000018       __imp_ShowWindow           0011b018     coredll:COREDLL.dll
 0003:0000001c       __imp_SetWindowTextW       0011b01c     coredll:COREDLL.dll
 0003:00000020       __imp_wcscat               0011b020     coredll:COREDLL.dll
 0003:00000024       __imp_LoadStringW          0011b024     coredll:COREDLL.dll
 0003:00000028       __imp_MessageBoxW          0011b028     coredll:COREDLL.dll
 0003:0000002c       __imp_GetLastError         0011b02c     coredll:COREDLL.dll
 0003:00000030       __imp_CreateProcessW       0011b030     coredll:COREDLL.dll
 0003:00000034       __imp_SetFocus             0011b034     coredll:COREDLL.dll
 0003:00000038       __imp_EndDialog            0011b038     coredll:COREDLL.dll
 0003:0000003c       __imp_DialogBoxIndirectParamW 0011b03c     coredll:COREDLL.dll
 0003:00000040       __imp_LoadResource         0011b040     coredll:COREDLL.dll
 0003:00000044       __imp_FindResourceW        0011b044     coredll:COREDLL.dll
 0003:00000048       __imp_swprintf             0011b048     coredll:COREDLL.dll
 0003:0000004c       __imp_RegisterClassW       0011b04c     coredll:COREDLL.dll
 0003:00000050       __imp_GetStockObject       0011b050     coredll:COREDLL.dll
 0003:00000054       __imp_memset               0011b054     coredll:COREDLL.dll
 0003:00000058       __imp_RegisterWindowMessageW 0011b058     coredll:COREDLL.dll
 0003:0000005c       __imp_SetWindowPos         0011b05c     coredll:COREDLL.dll
 0003:00000060       __imp_GetClientRect        0011b060     coredll:COREDLL.dll
 0003:00000064       __imp_SendMessageW         0011b064     coredll:COREDLL.dll
 0003:00000068       __imp_SendDlgItemMessageW  0011b068     coredll:COREDLL.dll
 0003:0000006c       __imp_RegCloseKey          0011b06c     coredll:COREDLL.dll
 0003:00000070       __imp_NKDbgPrintfW         0011b070     coredll:COREDLL.dll
 0003:00000074       __imp_RegQueryValueExW     0011b074     coredll:COREDLL.dll
 0003:00000078       __imp_RegOpenKeyExW        0011b078     coredll:COREDLL.dll
 0003:0000007c       __imp_RegSetValueExW       0011b07c     coredll:COREDLL.dll
 0003:00000080       __imp_RegCreateKeyExW      0011b080     coredll:COREDLL.dll
 0003:00000084       __imp_wsprintfW            0011b084     coredll:COREDLL.dll
 0003:00000088       __imp__isctype             0011b088     coredll:COREDLL.dll
 0003:0000008c       __imp_wcslen               0011b08c     coredll:COREDLL.dll
 0003:00000090       __imp_GetWindowTextW       0011b090     coredll:COREDLL.dll
 0003:00000094       __imp_KillTimer            0011b094     coredll:COREDLL.dll
 0003:00000098       __imp_TlsGetValue          0011b098     coredll:COREDLL.dll
 0003:0000009c       __imp_malloc               0011b09c     coredll:COREDLL.dll
 0003:000000a0       __imp_WideCharToMultiByte  0011b0a0     coredll:COREDLL.dll
 0003:000000a4       __imp_free                 0011b0a4     coredll:COREDLL.dll
 0003:000000a8       __imp_strcpy               0011b0a8     coredll:COREDLL.dll
 0003:000000ac       __imp_memcpy               0011b0ac     coredll:COREDLL.dll
 0003:000000b0       __imp_LoadLibraryW         0011b0b0     coredll:COREDLL.dll
 0003:000000b4       __imp_GetWindowRect        0011b0b4     coredll:COREDLL.dll
 0003:000000b8       __imp_SetWindowLongW       0011b0b8     coredll:COREDLL.dll
 0003:000000bc       __imp_GetWindowLongW       0011b0bc     coredll:COREDLL.dll
 0003:000000c0       __imp_OutputDebugStringW   0011b0c0     coredll:COREDLL.dll
 0003:000000c4       __imp_wvsprintfW           0011b0c4     coredll:COREDLL.dll
 0003:000000c8       __imp_??3@YAXPAX@Z         0011b0c8     coredll:COREDLL.dll
 0003:000000cc       __imp_??2@YAPAXI@Z         0011b0cc     coredll:COREDLL.dll
 0003:000000d0       __imp_memcmp               0011b0d0     coredll:COREDLL.dll
 0003:000000d4       __imp_GetModuleFileNameW   0011b0d4     coredll:COREDLL.dll
 0003:000000d8       __imp_GetModuleHandleW     0011b0d8     coredll:COREDLL.dll
 0003:000000dc       __imp_RegDeleteKeyW        0011b0dc     coredll:COREDLL.dll
 0003:000000e0       __imp__purecall            0011b0e0     coredll:COREDLL.dll
 0003:000000e4       __imp_PostMessageW         0011b0e4     coredll:COREDLL.dll
 0003:000000e8       __imp_RemoveProp           0011b0e8     coredll:COREDLL.dll
 0003:000000ec       __imp_GetActiveWindow      0011b0ec     coredll:COREDLL.dll
 0003:000000f0       __imp_wcscpy               0011b0f0     coredll:COREDLL.dll
 0003:000000f4       __imp_DefWindowProcW       0011b0f4     coredll:COREDLL.dll
 0003:000000f8       __imp_EndPaint             0011b0f8     coredll:COREDLL.dll
 0003:000000fc       __imp_DrawTextW            0011b0fc     coredll:COREDLL.dll
 0003:00000100       __imp_ExtTextOutW          0011b100     coredll:COREDLL.dll
 0003:00000104       __imp_BeginPaint           0011b104     coredll:COREDLL.dll
 0003:00000108       __imp_InvalidateRect       0011b108     coredll:COREDLL.dll
 0003:0000010c       __imp_CreateWindowExW      0011b10c     coredll:COREDLL.dll
 0003:00000110       __imp_TlsCall              0011b110     coredll:COREDLL.dll
 0003:00000114       __imp_CreateThread         0011b114     coredll:COREDLL.dll
 0003:00000118       __imp_LoadIconW            0011b118     coredll:COREDLL.dll
 0003:0000011c       __imp_DestroyIcon          0011b11c     coredll:COREDLL.dll
 0003:00000120       __imp_wcsncpy              0011b120     coredll:COREDLL.dll
 0003:00000124       __imp___rt_sdiv            0011b124     coredll:COREDLL.dll
 0003:00000128       __imp_InterlockedCompareExchange 0011b128     coredll:COREDLL.dll
 0003:0000012c       __imp_SetTimer             0011b12c     coredll:COREDLL.dll
 0003:00000130       __imp_Sleep                0011b130     coredll:COREDLL.dll
 0003:00000134       __imp_LocalAlloc           0011b134     coredll:COREDLL.dll
 0003:00000138       __imp_TlsSetValue          0011b138     coredll:COREDLL.dll
 0003:0000013c       __imp_memmove              0011b13c     coredll:COREDLL.dll
 0003:00000140       __imp_?terminate@std@@YAXXZ 0011b140     coredll:COREDLL.dll
 0003:00000144       __imp___C_specific_handler 0011b144     coredll:COREDLL.dll
 0003:00000148       __imp_strcmp               0011b148     coredll:COREDLL.dll
 0003:0000014c       __imp___security_gen_cookie 0011b14c     coredll:COREDLL.dll
 0003:00000150       __imp_LocalFree            0011b150     coredll:COREDLL.dll
 0003:00000154       __imp___report_gsfailure   0011b154     coredll:COREDLL.dll
 0003:00000158       \177COREDLL_NULL_THUNK_DATA 0011b158     coredll:COREDLL.dll
 0003:0000015c       __imp_UIMUnblockPIN        0011b15c     gobiapi:GobiApi.dll
 0003:00000160       __imp_UIMSetPINProtection  0011b160     gobiapi:GobiApi.dll
 0003:00000164       __imp_UIMVerifyPIN         0011b164     gobiapi:GobiApi.dll
 0003:00000168       __imp_UIMChangePIN         0011b168     gobiapi:GobiApi.dll
 0003:0000016c       __imp_UIMGetCardStatus     0011b16c     gobiapi:GobiApi.dll
 0003:00000170       __imp_QCWWANDisconnect     0011b170     gobiapi:GobiApi.dll
 0003:00000174       __imp_QCWWANConnect        0011b174     gobiapi:GobiApi.dll
 0003:00000178       __imp_SwiSetDeviceRemovalCallback 0011b178     gobiapi:GobiApi.dll
 0003:0000017c       __imp_GetCDMANetworkParameters 0011b17c     gobiapi:GobiApi.dll
 0003:00000180       __imp_SetCDMANetworkParameters 0011b180     gobiapi:GobiApi.dll
 0003:00000184       __imp_GetRTREConfig        0011b184     gobiapi:GobiApi.dll
 0003:00000188       \177GobiApi_NULL_THUNK_DATA 0011b188     gobiapi:GobiApi.dll
 0003:0000018c       __imp_tapiRequestMakeCallW 0011b18c     cellcore:cellcore.dll
 0003:00000190       \177cellcore_NULL_THUNK_DATA 0011b190     cellcore:cellcore.dll
 0003:00000194       __imp_DestroyPropertySheetPage 0011b194     commctrl:commctrl.dll
 0003:00000198       __imp_CreatePropertySheetPageW 0011b198     commctrl:commctrl.dll
 0003:0000019c       \177commctrl_NULL_THUNK_DATA 0011b19c     commctrl:commctrl.dll
 0003:000001a0       __imp_?SetAutoUpdateTime@@YAXH@Z 0011b1a0     sw_utilityG:sw_utilityG.dll
 0003:000001a4       __imp_?GetAutoUpdateTimeUI@@YAKXZ 0011b1a4     sw_utilityG:sw_utilityG.dll
 0003:000001a8       __imp_?GetAutoUpdateTime@@YAKXZ 0011b1a8     sw_utilityG:sw_utilityG.dll
 0003:000001ac       __imp_?SetCallGuardReg@@YAXK@Z 0011b1ac     sw_utilityG:sw_utilityG.dll
 0003:000001b0       __imp_GetVersionInfo       0011b1b0     sw_utilityG:sw_utilityG.dll
 0003:000001b4       __imp_?GetCallGuardReg@@YAKXZ 0011b1b4     sw_utilityG:sw_utilityG.dll
 0003:000001b8       __imp_?InitLog@@YAXPAUHINSTANCE__@@@Z 0011b1b8     sw_utilityG:sw_utilityG.dll
 0003:000001bc       __imp_?GetVerInfo@@YAPAGPAUHINSTANCE__@@@Z 0011b1bc     sw_utilityG:sw_utilityG.dll
 0003:000001c0       __imp_?LogV@@YAXPBGZZ      0011b1c0     sw_utilityG:sw_utilityG.dll
 0003:000001c4       __imp_ModGetPreferredPrivacyMode 0011b1c4     sw_utilityG:sw_utilityG.dll
 0003:000001c8       __imp_ModGetRoamStatus     0011b1c8     sw_utilityG:sw_utilityG.dll
 0003:000001cc       __imp_ModGetLocationStatus 0011b1cc     sw_utilityG:sw_utilityG.dll
 0003:000001d0       __imp_ModGetRoamingMode    0011b1d0     sw_utilityG:sw_utilityG.dll
 0003:000001d4       __imp_ModSetRoamingMode    0011b1d4     sw_utilityG:sw_utilityG.dll
 0003:000001d8       __imp_ModSetPreferredPrivacyMode 0011b1d8     sw_utilityG:sw_utilityG.dll
 0003:000001dc       __imp_ModSetLocationMode   0011b1dc     sw_utilityG:sw_utilityG.dll
 0003:000001e0       __imp_GetRilStatus         0011b1e0     sw_utilityG:sw_utilityG.dll
 0003:000001e4       __imp_?LogW@@YAXPBGZZ      0011b1e4     sw_utilityG:sw_utilityG.dll
 0003:000001e8       __imp_?GetProductFeatures@@YAHAAK@Z 0011b1e8     sw_utilityG:sw_utilityG.dll
 0003:000001ec       __imp_SetEquipmentState    0011b1ec     sw_utilityG:sw_utilityG.dll
 0003:000001f0       __imp_?InWideMode@@YAHXZ   0011b1f0     sw_utilityG:sw_utilityG.dll
 0003:000001f4       __imp_?RelayoutDialog@@YAHPAUHINSTANCE__@@PAUHWND__@@PBG@Z 0011b1f4     sw_utilityG:sw_utilityG.dll
 0003:000001f8       __imp_GetOMADMConfig       0011b1f8     sw_utilityG:sw_utilityG.dll
 0003:000001fc       __imp_?LogStoreFileLine@@YAXPAGH@Z 0011b1fc     sw_utilityG:sw_utilityG.dll
 0003:00000200       __imp_?WriteLog@@YAXKPBGZZ 0011b200     sw_utilityG:sw_utilityG.dll
 0003:00000204       __imp_?LogC@@YAXPBGZZ      0011b204     sw_utilityG:sw_utilityG.dll
 0003:00000208       __imp_?SetConnectionProfile@@YAJXZ 0011b208     sw_utilityG:sw_utilityG.dll
 0003:0000020c       __imp_GetLogoTestReg       0011b20c     sw_utilityG:sw_utilityG.dll
 0003:00000210       __imp_?GetCarrierIndex@@YAKXZ 0011b210     sw_utilityG:sw_utilityG.dll
 0003:00000214       __imp_?SetNormalCursor@@YAXXZ 0011b214     sw_utilityG:sw_utilityG.dll
 0003:00000218       __imp_?SetWaitCursor@@YAXXZ 0011b218     sw_utilityG:sw_utilityG.dll
 0003:0000021c       \177sw_utilityG_NULL_THUNK_DATA 0011b21c     sw_utilityG:sw_utilityG.dll
 0003:00000220       __xc_a                     0011b220     corelibc:crt0init.obj
 0003:0000026c       __xc_z                     0011b26c     corelibc:crt0init.obj
 0003:00000270       __xi_a                     0011b270     corelibc:crt0init.obj
 0003:00000274       __xi_z                     0011b274     corelibc:crt0init.obj
 0003:00000278       __xp_a                     0011b278     corelibc:crt0init.obj
 0003:0000027c       __xp_z                     0011b27c     corelibc:crt0init.obj
 0003:00000280       __xt_a                     0011b280     corelibc:crt0init.obj
 0003:00000284       __xt_z                     0011b284     corelibc:crt0init.obj
 0003:00000288       ?g_szDataClass@@3PAGA      0011b288     data.obj
 0003:0000028c       ?g_szDatalistClass@@3PAGA  0011b28c     datalist.obj
 0003:00000290       ?g_szLocationClass@@3PAGA  0011b290     location.obj
 0003:00000294       ?g_szPhsListClass@@3PAGA   0011b294     phs_list.obj
 0003:0000029c       ?g_sz_RUIM_CALL_CTRL_DlgClass@@3PAGA 0011b29c     ruim_call_ctrl.obj
 0003:000002a4       ?g_sz_RUIM_PIN_DlgClass@@3PAGA 0011b2a4     ruim_pin.obj
 0003:000002a8       ?PinStateText@@3PAPAGA     0011b2a8     ruim_pin.obj
 0003:000002c4       ?g_sz_SPRINT_ROAMING_OPTION_DlgClass@@3PAGA 0011b2c4     Sprint_roaming_option.obj
 0003:000002c8       ?MY_NOTIFYICON@@3IA        0011b2c8     sw_emext.obj
 0003:000002cc       ?g_szSysSettingsClass@@3PAGA 0011b2cc     syssettings.obj
 0003:000002d4       ?g_szVersionInfoDlgClass@@3PAGA 0011b2d4     versioninfo.obj
 0003:000002d8       __security_cookie_complement 0011b2d8     corelibc:seccook.obj
 0003:000002dc       __security_cookie          0011b2dc     corelibc:seccook.obj
 0003:000002ec       ?g_hWndDataList@@3PAUHWND__@@A 0011b2ec     datalist.obj
 0003:000002f0       ?g_bProvision@@3HA         0011b2f0     datalist.obj
 0003:000002f4       ?g_bReset@@3HA             0011b2f4     datalist.obj
 0003:000002fc       ?g_hWndPhsList@@3PAUHWND__@@A 0011b2fc     phs_list.obj
 0003:00000300       ?g_hWndMainList@@3PAUHWND__@@A 0011b300     phs_list.obj
 0003:00000308       ?g_CallCrlTimer@@3IA       0011b308     ruim_call_ctrl.obj
 0003:00000318       ?gPIN1State@@3EA           0011b318     ruim_pin.obj
 0003:0000031c       ?gDialog@@3PAUHWND__@@A    0011b31c     ruim_pin.obj
 0003:00000348       ?g_szBuffer@@3PAGA         0011b348     sw_emext.obj
 0003:000012e8       ?g_hCurrentWnd@@3PAUHWND__@@A 0011c2e8     sw_emext.obj
 0003:000012ec       ?g_nCarrier@@3KA           0011c2ec     sw_emext.obj
 0003:000012f0       ?g_Err@@3UtagErrorInfo@@A  0011c2f0     sw_emext.obj
 0003:000014f8       ?g_stRilStatus@@3USW_RILStatus@@A 0011c4f8     sw_emext.obj
 0003:00001538       ?g_hResInst@@3PAUHINSTANCE__@@A 0011c538     sw_emext.obj
 0003:0000153c       ?g_hInst@@3PAUHINSTANCE__@@A 0011c53c     sw_emext.obj
 0003:00001540       ?g_dwDLLRefCount@@3IA      0011c540     sw_emext.obj
 0003:00001544       ?g_hwndERI@@3PAUHWND__@@A  0011c544     sw_emext.obj
 0003:00001548       ?g_dwLen@@3KA              0011c548     sw_emext.obj
 0003:0000154c       ?gGobiConnected@@3HA       0011c54c     sw_emext.obj
 0003:00001550       ?g_RUIMRefreshTimer@@3IA   0011c550     sw_emext.obj
 0003:00001554       ?g_RoamRefreshTimer@@3IA   0011c554     sw_emext.obj
 0003:00001558       ?g_DeviceSearchTimer@@3IA  0011c558     sw_emext.obj
 0003:0000155c       ?g_hIconDormant@@3PAUHICON__@@A 0011c55c     sw_emext.obj
 0003:00001560       ?g_hIconRevA@@3PAUHICON__@@A 0011c560     sw_emext.obj
 0003:00001564       ?g_hDlg@@3PAUHWND__@@A     0011c564     sw_emext.obj
 0003:00001578       ?g_VersionInfo@@3UtagRILVERNOINFO@@A 0011c578     versioninfo.obj
 0003:00002188       __onexitend                0011d188     <common>
 0003:0000218c       __onexitbegin              0011d18c     <common>
 0003:00002190       _exitflag                  0011d190     <common>
 0003:00002194       _pRawDllMain               0011d194     <common>

 entry point at        0001:0000f934

 Static symbols

 0001:000057f8       __unwind$41605             001067f8 f   ruim_pin.obj
 0001:00005818       __unwind$41606             00106818 f   ruim_pin.obj
 0001:00005838       __unwind$41607             00106838 f   ruim_pin.obj
 0001:00005858       __unwind$41608             00106858 f   ruim_pin.obj
 0001:00005878       __unwind$41609             00106878 f   ruim_pin.obj
 0001:00005bb4       __unwind$41687             00106bb4 f   ruim_pin.obj
 0001:00005bd4       __unwind$41688             00106bd4 f   ruim_pin.obj
 0001:00007edc       ?WriteDWORDValue@@YAJPAUHKEY__@@PBG1K@Z 00108edc f   Sprint_roaming_option.obj
 0001:00008460       ?ReadDWORDValue@@YAJPAUHKEY__@@PBG1PAK@Z 00109460 f   Sprint_roaming_option.obj
 0001:0000899c       __unwind$42438             0010999c f   sw_emext.obj
 0001:00009de4       ?DeviceRemovalCallback@@YAXK@Z 0010ade4 f   sw_emext.obj
 0001:0000fa2c       _initterm                  00110a2c f   corelibc:crt0dat.obj
 0001:0000facc       doexit                     00110acc f   corelibc:crt0dat.obj
 0001:0000ff88       ?FindHandler@@YAEPAUEHExceptionRecord@@PAKPAU_CONTEXT@@PAU_DISPATCHER_CONTEXT@@PBU_s_FuncInfo@@H@Z 00110f88 f   LIBCMTD:frame_ce.obj
 0001:0001057c       ?TypeMatch@@YAHPBU_s_HandlerType@@PBU_s_CatchableType@@PBU_s_ThrowInfo@@@Z 0011157c f   LIBCMTD:frame_ce.obj
 0001:00010940       ?FrameUnwindFilter@@YAHPAU_EXCEPTION_POINTERS@@@Z 00111940 f   LIBCMTD:frame_ce.obj
 0001:000109cc       ?CallCatchBlock@@YAPAXPAUEHExceptionRecord@@PAKPAU_CONTEXT@@PBU_s_FuncInfo@@PAXHK@Z 001119cc f   LIBCMTD:frame_ce.obj
 0001:00010f68       ?CanThisExceptionObjectBeDestructed@@YAEPAUEHExceptionRecord@@E@Z 00111f68 f   LIBCMTD:frame_ce.obj
 0001:000111f4       ?BuildCatchObject@@YAXPAUEHExceptionRecord@@PAKPBU_s_HandlerType@@PBU_s_CatchableType@@@Z 001121f4 f   LIBCMTD:frame_ce.obj
 0001:00011544       ?AdjustPointer@@YAPAXPAXABUPMD@@@Z 00112544 f   LIBCMTD:frame_ce.obj
 0001:00011e48       ??__ERIL_STATUS_CHANGED@@YAXXZ 00112e48 f   data.obj
 0001:00011e78       ??__ERIL_STATUS_CHANGED@@YAXXZ 00112e78 f   location.obj
 0001:00011ea8       ??__ERIL_STATUS_CHANGED@@YAXXZ 00112ea8 f   ruim_call_ctrl.obj
 0001:00011ed8       ??__ERIL_DBG_NOTIFY@@YAXXZ 00112ed8 f   ruim_call_ctrl.obj
 0001:00011f08       ??__ERIL_SET_ERITEXT@@YAXXZ 00112f08 f   ruim_call_ctrl.obj
 0001:00011f38       ??__ERIL_STATUS_CHANGED@@YAXXZ 00112f38 f   ruim_pin.obj
 0001:00011f68       ??__ERIL_DBG_NOTIFY@@YAXXZ 00112f68 f   ruim_pin.obj
 0001:00011f98       ??__ERIL_SET_ERITEXT@@YAXXZ 00112f98 f   ruim_pin.obj
 0001:00011fc8       ??__ERIL_STATUS_CHANGED@@YAXXZ 00112fc8 f   Sprint_roaming_option.obj
 0001:00011ff8       ??__ERIL_DBG_NOTIFY@@YAXXZ 00112ff8 f   Sprint_roaming_option.obj
 0001:00012028       ??__ERIL_SET_ERITEXT@@YAXXZ 00113028 f   Sprint_roaming_option.obj
 0001:00012058       ??__ERIL_STATUS_CHANGED@@YAXXZ 00113058 f   stdafx.obj
 0001:00012088       ??__ERIL_DBG_NOTIFY@@YAXXZ 00113088 f   stdafx.obj
 0001:000120b8       ??__ERIL_SET_ERITEXT@@YAXXZ 001130b8 f   stdafx.obj
 0001:000120e8       ??__ERIL_STATUS_CHANGED@@YAXXZ 001130e8 f   sw_emext.obj
 0001:00012118       ??__ERIL_SET_ERITEXT@@YAXXZ 00113118 f   sw_emext.obj
 0001:00012148       ??__ERIL_STATUS_CHANGED@@YAXXZ 00113148 f   syssettings.obj
